:1000000017C026C025C024C08DC022C021C020C07A
:100010001FC01EC01DC01CC01BC01AC019C00037A5
:10002000003600380101010101010102040810201D
:1000300011241FBECFE5D2E0DEBFCDBF20E0A0E699
:10004000B0E001C01D92A936B207E1F7B2D090C16D
:10005000D7CFEBE2F0E09491E5E2F0E0E491EE231B
:1000600091F02AB52F7C2ABDF0E0EE5DFF4FA49100
:10007000B0E0811109C08FB7F8942C91E92FE09579
:10008000E223EC938FBF08958FB7F894EC91E92B9E
:10009000F8CF3FB7F8948091650090916600A091E9
:1000A0006700B09168002FB508B602FE05C02F3F6B
:1000B00019F00196A11DB11D3FBFBA2FA92F982F8E
:1000C0008827BC01CD01620F711D811D911D42E089
:1000D000660F771F881F991F4A95D1F70895CF9211
:1000E000DF92EF92FF92CF93DF936B017C01D1DF20
:1000F000EB01CFDF6C1B7D0B683E7340D0F381E0DA
:10010000C81AD108E108F108C851DC4FC114D10464
:10011000E104F10471F7DF91CF91FF90EF90DF9050
:10012000CF90089578941F920F920FB60F921124DA
:100130002F933F938F939F93AF93BF9380916100D1
:1001400090916200A0916300B091640030916000D2
:100150002CE7230F2D3728F02FEF230F0196A11D39
:10016000B11D209360008093610090936200A09382
:100170006300B09364008091650090916600A09147
:100180006700B09168000196A11DB11D80936500C4
:1001900090936600A0936700B0936800BF91AF9101
:1001A0009F918F913F912F910F900FBE0F901F90B5
:1001B0001895789480B7806880BF80B7806480BFCE
:1001C0008CB580648CBD8FEF8DBD80B7807F8760DC
:1001D00080BF89B7846089BF83B7887F83BF8AB5B2
:1001E0008C7F81608ABD83B7877F83BF83B7887F19
:1001F000836083BF86B1876086B9379A8FE2A82E65
:1002000080E0B82EF501249109E210E0F801849114
:10021000882391F090E0FC01E25EFF4FE491AE2F65
:10022000B0E0FC01EE5DFF4FE4918FB7F8949C9134
:10023000209529232C938FBFEBE2F0E02491E5E297
:10024000F0E0E491EE2389F08E2F90E0FC01E25E75
:10025000FF4FA491B0E08E5D9F4FFC0184918FB75A
:10026000F894EC91E22BEC938FBF81E0F2DE68EE24
:1002700073E080E090E033DF80E0EBDEF501349165
:10028000F801249180E090E0DC01E22FF0E0E05EF4
:10029000FF4F449150E0EA012881232331F144913A
:1002A00050E0EA012881232361F5C12CD12C76018D
:1002B000449150E0EA012881232379F128E032E5D6
:1002C00040E050E0C701B6013AD06058714C8F4F02
:1002D0009F4F643770448105910508F4CFCF64E6E1
:1002E00070E080E090E0FBDEC0CF0196A11DB11D63
:1002F000883922E7920723E0A207B10509F0C9CFA8
:10030000BDCF0196A11DB11D8839D2E79D07D3E06D
:10031000AD07B10509F0C3CFB1CFAC01BD014C0DA4
:100320005D1D6E1D7F1D473952476340710509F4FD
:10033000A5CF2FEFC21AD20AE20AF20AB9CFEE27EE
:10034000FF27AA27BB2708C0A20FB31FE41FF51F72
:10035000220F331F441F551F9695879577956795F4
:1003600098F37040A9F7009799F7BD01CF01089560
:04037000F894FFCF2F
:00000001FF
